:020000040000FA
:02000000AC2929
:08000800831203138601831229
:10001000031385018312031341190616C1198616AD
:10002000411A0617C11A8617640083120313E00AE7
:10003000031D142883120313F50A031D142803015A
:10004000830183120313851386100611051483128E
:1000500003138B102621640083120313061C2B2824
:1000600044213921CF2983120313C008031D08003E
:10007000831203138614E73083120313C000023087
:1000800083120313C300080083120313C008031D67
:100090000800831203138610E73083120313C00095
:1000A000013083120313C3000800C40A031D0800B3
:1000B000C00A080083120313861E6B28FC308312CB
:1000C0000313C600FD3083120313E600FC308312D5
:1000D0000313E900912883120313061F7C28FC30C8
:1000E00083120313C600FD3083120313E600FC30B5
:1000F00083120313E900912883120313861F8D28AE
:10010000FC3083120313C600FD3083120313E60094
:10011000FC3083120313E9009128FD30831203138E
:10012000C6009C3083120313E10083120313571897
:10013000AA2883120313F40A031D08008312031371
:10014000E10A0319A42808008312031386158312F9
:100150000313571483120313F20A031D08008312BA
:100160000313F30A031D080083120313C60A0800D1
:10017000831203130619E52883120313C80A031D0B
:10018000080083120313F10A031D080083120313EE
:10019000051483120313D50A031D0800E5288312F2
:1001A00003130619E52883120313C80A031D080068
:1001B00083120313F10A031D0800831203130514AD
:1001C00083120313F00A031D080083120313061D94
:1001D000EB289520080006155A2008008312031307
:1001E0000611051083120313D714571057138312E7
:1001F00003134110C11408008312031306110510E4
:10020000831203135715571057138312031341100A
:10021000C11408008312031306110510831203137F
:10022000D71557105713831203134110C114080038
:100230008312031306110510831203135716571068
:100240005713831203134110C114080083120313C0
:1002500085170615442183120313851306114421C3
:100260008312031306154421831203138513061109
:1002700009008513442183120313061544218312B8
:100280000313851306110900383083120313D900B4
:10029000640083120313D80A031D48298312031331
:1002A000D90A031D4829080083120313E20A031D1B
:1002B000080083120313E30A031D080083120313CB
:1002C0008611831203135717080083120313E40ADD
:1002D000031D080083120313E50A031D080083129F
:1002E0000313E60A031D0800831203130517831284
:1002F00003135713080083120313E70A031D0800B2
:1003000083120313E80A031D080083120313E90A8A
:10031000031D08008312031305130800831203133F
:10032000851E080083120313C11897290800831241
:100330000313F70A031D080083120313F80A031DB1
:10034000080083120313F90A031D08008312031324
:10035000C20A031D0800AB2983120313061283127D
:100360000313D7018312031385018312031386013C
:10037000831203138301BC2983163E3085000130AC
:1003800086008C308100831207309F00083083166E
:1003900003138E00D030831203138B002B2883129B
:1003A0000313D701831203138501831203138601FC
:1003B00083120313D71683120313E7018312031367
:1003C000E80183120313E40183120313E50183128E
:1003D0000313F10183120313F20183120313F301D8
:1003E00083120313F40183120313C1018312031355
:1003F000F70183120313F80183120313F901831227
:100400000313C201003083120313E2009C308312F5
:100410000313E300FC3083120313E600FC30831265
:100420000313E9002B3083120313F900E730831222
:100430000313C20083120313851383120313861060
:1004400083120313830183120313C4018312031362
:10045000C50183120313C80183120313D801FF30AF
:1004600083120313D500CE3083120313F100FD3045
:1004700083120313F00083120313C70183120313C3
:10048000C001013083120313C300FF308312031332
:10049000C600013083120313430203193320831271
:1004A0000313411C572A83120313061E7B2A83124F
:1004B00003135718542183120313571B652183120A
:1004C0000313051B7B2183120313D7187B2A85187E
:1004D0000616061E7B2A8312031341144115CF20F2
:1004E000C6080319EE2083120313411C7B2A8312D2
:1004F0000313861E9F2A8312031357185421831255
:100500000313571B652183120313051B7B218312E1
:10051000031357199F2A05198616861E9F2A8312D0
:1005200003134114C115B820C6080319FC20831217
:100530000313411C9F2A83120313061FC32A83122D
:1005400003135718542183120313571B6521831279
:100550000313051B7B2183120313D719C32A8519A3
:100560000617061FC32A8312031341144116B8202D
:10057000C60803190A2183120313411CC32A8312DC
:100580000313861FDF2A8312031357185421831283
:100590000313571B652183120313051B7B21831251
:1005A0000313571ADF2A051A8617861FDF2A8312BC
:1005B00003134114C116B820C608031918210230CC
:1005C0008312031343020319442055208E21640033
:0205D000492AB6
:02400E00543F1D
:00000001FF
